:100000000C94B3060C94FA060C94FA060C94FA06B7
:100010000C94FA060C94FA060C94FA060C94FA0660
:100020000C94FA060C94FA060C9400160C94D21652
:100030000C94A9250C94FA060C94FA060C94FA0672
:100040000C94FA060C94FA060C94FA060C94FA0630
:100050000C94FA060C9449260C94FA060C94FA06B1
:100060000C94FA060C9447090C94FA060C94FA06C0
:100070000C94FA060C94FA060C94FA060C94FA0600
:100080000C94FA060C94FA060C94FA060C94FA06F0
:100090000C94FA060C94FA060C94FA060C94FA06E0
:1000A0000C94FA060C94FA060C94FA06850E890E46
:1000B0008D0E910E950E990E9D0EA10EA50EA90EF8
:1000C000AD0EB10EB50EB90EBD0EC10EC50EC90EE8
:1000D000CD0ED10ED50ED90EDD0EE10EE50EE90ED8
:1000E000ED0EF10EF50EF90EFD0E010F050F090FC5
:1000F0000D0F110F510F830E150F170F190F1B0F37
:100100001F0F230F270F2B0F300F350F390F3D0F08
:10011000410F450F490F4F0F4F0F4F0F4F0F4F0F0D
:100120004F0F4F0F4F0F4F0F4F0F4F0F4F0F4F0FDF
:100130004F0F4F0F4F0F4F0F4F0F4F0F4D0F3F17D9
:1001400061174F1861174F18A617C9174F181E18B7
:100150003118311B311B601B601BBE1BFC1B161EA4
:10016000161E151C161E161D161DEA1D161E161E21
:10017000011E1F141A16041D1B062021150807094D
:10018000190522231C170A0B11801E352B39797A89
:100190007B2C2425180C0E0D1080742A31287C7DB0
:1001A0007E7F26271213330F36802D2E302F3438C2
:1001B000378025630025730D0A00522C310D0A008B
:1001C00053592C464646340D0A0053482C303033E0
:1001D000430D0A00537E2C360D0A0053572C38303D
:1001E00030300D0A00534D2C340D0A0053532C4B64
:1001F0006579626F6172642F4D6F7573650D0A00CA
:10020000532D2C546D6B42540D0A0053462C310D66
:100210000A002D2D2D0D0A0045786974696E67203E
:10022000636F6E666967206D6F6465202E2E2E0ADF
:10023000002B0D0A00760D0A0024242400456E745C
:100240006572696E6720636F6E666967206D6F64A3
:1002500065202E2E2E0A00522C310D0A0053522CEE
:100260005A0D0A00555342206D6F64650A004175AE
:10027000746F206D6F64650A00253032750A0025A1
:100280003032753A00253032753A004241543A20F6
:1002900025756D560900757074696D653A202530B5
:1002A000327520253032753A253032753A25303294
:1002B000750A00564255533A2025580A0052656D7A
:1002C0006F746557616B657570456E61626C6564CE
:1002D0003A2025580A000A003F004C4F5700444975
:1002E000534348470043484152470046554C4C0051
:1002F000626174746572793A2000555342205374D8
:100300006174653A2025730A00636F6E6669675FE2
:100310006D6F64653A2025580A00726E34325F6151
:1003200075746F636F6E6E656374696E6728293AC2
:100330002025580A00726E34323A2025730A00666E
:100340006F7263655F7573623A2025580A00707298
:100350006F746F636F6C3A2025730A000A2D2D2D80
:100360002D2D20524E2D343220696E666F202D2D9A
:100370002D2D2D0A00753A20202020202020746F7A
:1003800067676C6520466F72636520555342206D28
:100390006F64650A00703A202020202020207061C0
:1003A0006972696E670A00536C636B3A20202020E3
:1003B000524E2D343220696E697469616C697A65B8
:1003C0000A0044656C3A2020202020656E74657216
:1003D0002F6578697420524E2D343220636F6E661B
:1003E0006967206D6F64650A00623A202020202032
:1003F00020206261747465727920766F6C74616715
:10040000650A00693A20202020202020524E2D34F9
:100410003220696E666F0A000A0A2D2D2D2D2D20BF
:10042000426C7565746F6F746820524E2D343220A3
:1004300048656C70202D2D2D2D2D0A00253032752C
:100440003A253032753A253032750925756D560AD0
:10045000004C4544207374617475733A2025303222
:10046000580A002025303258002563005B735D0078
:100470004B6579626F6172642073746172740A00F3
:10048000524E2D343220696E69740A000A55534267
:1004900020696E69740A005B445D005B435D001275
:1004A00003480048004B00420020006D006F0064CC
:1004B0000000000E0374002E006D002E006B002E55
:1004C0000000000403090409028D00050100A032A8
:1004D00009040000010301010009211101000122AA
:1004E00040000705810308000A0904010001030117
:1004F0000200092111010001224D000705820308B5
:10050000000A090402000103000000092111010092
:10051000012236000705830308000A0904030002CC
:1005200003000000092111010001222200070584B7
:100530000320000107050403200001090404000151
:10054000030000000921110100012239000705857F
:10055000032000011201100100000008EDFE4242DC
:1005600004010102000105010906A101050719E0C6
:1005700029E7150025019508750181020508190173
:1005800029059505750191029501750391010507EE
:10059000190029F71500250195F875018102C0069B
:1005A00031FF0974A1010975150026FF009520751A
:1005B0000881020976150026FF0095207508910232
:1005C000C005010980A101850216810026B7001A25
:1005D00081002AB700751095018100C0050C090142
:1005E000A1018503160100269C021A01002A9C0223
:1005F000751095018100C005010902A1010901A141
:1006000000050919012905150025019505750181C8
:100610000295017503810105010930093115812514
:100620007F95027508810609381581257F9501752A
:10063000088106050C0A38021581257F9501750889
:100640008106C0C005010906A101050719E029E7D7
:100650001500250195087501810295017508810134
:100660000508190129059505750191029501750384
:1006700091010507190029FF150026FF0095067551
:10068000088100C0636F6E73756D65723A20253006
:1006900034580A0073797374656D3A2025303458E4
:1006A0000A000A002530325820006B6579626F61BC
:1006B00072643A20004C45443A20253032580A00F2
:1006C000253032583A202530386225730A00722FBF
:1006D000632030313233343536370A0064656C5F5D
:1006E0006B65795F6269743A2063616E2774206478
:1006F000656C3A20253032580A006164645F6B658E
:10070000795F6269743A2063616E27742061646462
:100710003A20253032580A004F6E6573686F743A7C
:100720002074696D656F75740A00290A00257500CB
:100730002F002575005D2800256400200025640039
:10074000200025640020002564007C0025303258FC
:10075000006D6F7573656B6579205B62746E7C7874
:100760002079207620685D287265702F61636C297E
:100770003A205B006D6B5F776865656C5F74696DCF
:10078000655F746F5F6D6178203D2025640A006DA0
:100790006B5F776865656C5F6D61785F73706565C9
:1007A00064203D2025640A006D6B5F74696D655F90
:1007B000746F5F6D6178203D2025640A006D6B5F6A
:1007C0006D61785F7370656564203D2025640A0063
:1007D0006D6B5F696E74657276616C203D20256477
:1007E0000A006D6B5F64656C6179203D2025640AA9
:1007F000006D6B5F776865656C5F74696D655F74CC
:100800006F5F6D6178203D2025640A006D6B5F7716
:100810006865656C5F6D61785F7370656564203DC8
:100820002025640A006D6B5F74696D655F746F5F8E
:100830006D6178203D2025640A006D6B5F6D6178E5
:100840005F7370656564203D2025640A006D6B5FF1
:10085000696E74657276616C203D2025640A006DB6
:100860006B5F64656C6179203D2025640A000A0095
:10087000257500363A20776865656C5F74696D652B
:100880005F746F5F6D61783A20000A00257500354E
:100890003A20776865656C5F6D61785F7370656538
:1008A000643A20000A00257500343A2074696D65A9
:1008B0005F746F5F6D61783A20000A002575003320
:1008C0003A206D61785F73706565643A20000A00B4
:1008D000257500323A20696E74657276616C286DF8
:1008E00073293A20000A00257500313A2064656CAE
:1008F0006179282A31306D73293A20000A092D20A8
:1009000056616C756573202D0A004D3E004D2564BF
:100910003E20003F007365742064656661756C74E9
:100920000A00433E200077686572652064656C7438
:10093000613A20637572736F723D25642C2077686D
:1009400065656C3D25640A53656520687474703A6A
:100950002F2F656E2E77696B6970656469612E6FE4
:1009600072672F77696B692F4D6F7573655F6B6564
:1009700079730A000A092D204D6F7573656B6579CF
:10098000202D0A4553432F713A09717569740A3154
:100990003A0964656C6179282A31306D73290A320D
:1009A0003A09696E74657276616C286D73290A3331
:1009B0003A096D61785F73706565640A343A097449
:1009C000696D655F746F5F6D61780A353A097768A4
:1009D00065656C5F6D61785F73706565640A363A52
:1009E00009776865656C5F74696D655F746F5F6DCD
:1009F00061780A0A703A097072696E742076616CC7
:100A00007565730A643A0973657420646566617577
:100A10006C74730A75703A092B310A646F776E3AF9
:100A2000092D310A706775703A092B31300A7067E9
:100A3000646F776E3A092D31300A0A737065656408
:100A4000203D2064656C7461202A206D61785F739D
:100A500070656564202A2028726570656174202F96
:100A60002074696D655F746F5F6D6178290A003F5E
:100A7000004D3E2000433E20004C25640A000A0938
:100A80002D20436F6E736F6C65202D0A4553432FE5
:100A9000713A09717569740A6D3A096D6F757365FC
:100AA0006B65790A000A092D204D61676963202D65
:100AB0000A643A0964656275670A783A096465628E
:100AC0007567206D61747269780A6B3A09646562B2
:100AD0007567206B6579626F6172640A6D3A0964AB
:100AE00065627567206D6F7573650A763A0976657C
:100AF0007273696F6E0A733A097374617475730A5D
:100B0000633A09636F6E736F6C65206D6F64650A7D
:100B1000302D343A096C61796572302D34284631B4
:100B2000302D4634290A506175733A09626F6F742B
:100B30006C6F616465720A6E3A094E4B524F0A003F
:100B40003F004E4B524F3A206F66660A004E4B52A2
:100B50004F3A206F6E0A0074696D65725F7265614D
:100B600064333228293A202530346C580A006B65EA
:100B700079626F6172645F6E6B726F3A2025580AFA
:100B8000006B6579626F6172645F69646C653A20BD
:100B900025580A006B6579626F6172645F70726FCD
:100BA000746F636F6C3A2025580A00686F73745F26
:100BB0006B6579626F6172645F6C65647328293A52
:100BC0002025580A000A092D20537461747573207A
:100BD0002D0A004743433A20342E392E3220415605
:100BE000522D4C4942433A20312E382E3073766EC6
:100BF000204156525F415243483A20617672350A8D
:100C0000004F5054494F4E533A204C554641204DC9
:100C10004F5553454B45592045585452414B455922
:100C200020434F4E534F4C4520434F4D4D414E4472
:100C3000204E4B524F204B45594D41505F53454339
:100C400054494F4E20343039360A004255494C44FD
:100C50003A2031623736656134202831383A3032F3
:100C60003A3430204D61722031362032303138290B
:100C70000A005649443A2030784645454428742EA7
:100C80006D2E6B2E29205049443A2030783432346E
:100C9000322848484B42206D6F6429205645523A0D
:100CA000203078303130340A00444553433A2074C0
:100CB0002E6D2E6B2E206B6579626F6172642066DB
:100CC00069726D7761726520666F722048484B4289
:100CD000206D6F640A000A092D2056657273696FD2
:100CE0006E202D0A000A6D6F7573653A206F666677
:100CF0000A000A6D6F7573653A206F6E0A000A6B01
:100D00006579626F6172643A206F66660A000A6BE9
:100D10006579626F6172643A206F6E0A000A6D61D4
:100D2000747269783A206F66660A000A6D6174729F
:100D300069783A206F6E0A000A64656275673A2026
:100D40006F6E0A000A64656275673A206F66660A0C
:100D5000000A0A626F6F746C6F616465722E2E2ECA
:100D60002000433E200011241FBECFEFDAE0DEBF9B
:100D7000CDBF04B603FE27C08091D6039091D70360
:100D8000A091D803B091D9038730904BA740B04BC6
:100D9000D1F41092D6031092D7031092D803109278
:100DA000D90314BE84B7877F84BF0FB6F894A89583
:100DB00080916000886180936000109260000FBE97
:100DC000E0E0F8E3099511E0A0E0B1E0E4EEFDE534
:100DD00002C005900D92A03AB107D9F723E0A0EA2E
:100DE000B1E001C01D92A63DB207E1F70E948C1050
:100DF0000C94F02E0C9400000FB680959AE0F894B5
:100E00007BE27A95F1F708F0589A08F4589886959D
:100E10009A95B1F70FBE08950FB680E8F894499BF4
:100E2000FECF4999FECF96E19A95F1F79CE29A950B
:100E3000F1F7869549998068C8F70FBE08950FB6F7
:100E400080E8F89496E19A95F1F79CE29A95F1F78B
:100E5000869549998068C8F796E19A95F1F7499B7C
:100E6000FECF0FBE0895FF93EF93E091A001F091A4
:100E7000A101309709F00995EF91FF910895FC01C8
:100E80008591803011F0EFDFFBCF0895FF27E0E27E
:100E900030E247FF0CC0419597FF09C0EDE2609535
:100EA000709580959095611D711D811D911D27FF85
:100EB00002C0219530E350E2AA27660F771F881FF2
:100EC000991FAA1FA41710F0A41B63955A95A9F7A0
:100ED000AA3008F0A95FA05DAF93F3956115710585
:100EE0008105910541F7ED3211F4EF93F395F21777
:100EF00018F43F93F395FBCF8F91B5DFFA95E1F7A7
:100F00000895E991F9918591803021F0853219F0A9
:100F1000AADFF9CF089520E0E89455915532C1F346
:100F2000503311F4689455915A3348F4505390F368
:100F3000220F022E220F220F200D250FF4CF0EF4C8
:100F4000219589919991533619F3533729F15335E6
:100F500059F1BC0188279927E8945C3621F48991DE
:100F6000999168945591543639F446EF7EF077FFA5
:100F70000DC08FEF9FEF0AC055374AE039F0583562
:100F800040E121F0523642E009F00895FF93EF93DB
:100F90007DDFEF91FF91B7CFFF93EF93FC0181913C
:100FA0008030B9F360DFFBCFFF93EF9368DFF1CFC1
:100FB000DF93CF93CDB7DEB72596A3DFCF91DF9137
:100FC000089514B88FEF85B9549A5C9808958FEFFF
:100FD00084B980E485B9549A5C9A8FE19EE40197C4
:100FE000F1F700C0000008958FEF84B980E485B95F
:100FF00057985F9A87B18F7387B988B1806C88B929
:101000002E9A2F980E94E107EAEAF1E088E08E0F1D
:1010100011928E13FDCFE2EAF1E088E08E0F11927B
:101020008E13FDCF8AEA91E09093B5018093B401CD
:1010300082EA91E09093B3018093B20108950F93F7
:101040001F93CF93DF938091B2019091B3012091D0
:10105000B4013091B5013093B3012093B201909364
:10106000B5018093B4015C9B0E94E707C0E0D0E02B
:1010700001E010E080E090E025B1207C2C2BAC0159
:1010800033E0440F551F3A95E1F7242B25B9EAE1E7
:10109000EA95F1F700C0E091B201F091B301EC0FD5
:1010A000FD1F208130E0082E02C0359527950A9457
:1010B000E2F720FD2F9AF5E3FA95F1F70000E6B587
:1010C0002E982AE12A95F1F700C04091B401509181
:1010D000B501DA01AC0FBD1F4F9B0AC09801082E65
:1010E00001C0220F0A94EAF720953C91232308C0FF
:1010F0006C919801082E01C0220F0A94EAF7262B62
:101100002C9326B56E2F70E02E1718F026B530E020
:1011100004C026B530E021503F4F261B370B263048
:10112000310558F0E091B201F091B301EC0FFD1FD1
:101130002081FA01EC0FFD1F20833AE13A95F1F787
:1011400000C02F982E9AEBE2F1E03197F1F700C042
:10115000000001968830910509F08ECFA091B4016E
:10116000B091B501AC0FBD1FE091B201F091B30198
:10117000EC0FFD1F9C918081981751F00E94E7258C
:101180006093B6017093B7018093B8019093B90151
:101190002196C830D10509F06DCF5C9B1BC08091B2
:1011A000CD03853021F08091CD03811113C0609172
:1011B000B6017091B7018091B8019091B9010E9478
:1011C0001D26613177428105910520F00E94E107DB
:1011D0000E94682581E0DF91CF911F910F910895C2
:1011E0002091B4013091B501F901E80FF11D808122
:1011F00008950C94E7070C94E107569A81FF02C00A
:101200005E9A08955E98089588E08093CC001092CD
:10121000CD00E9ECF0E08081806980838081886086
:101220008083EAECF0E080818083EBECF0E0808169
:101230008083559A5D98789408959091BB01209190
:10124000BA019217D1F030E0F901E454FE4F8081E9
:101250002F5F3F4F33272093BA01492F50E0921759
:1012600018F4241B350B03C0241B350B3395233096
:1012700031050CF05D9890E008958FEF9FEF089591
:101280009091C80095FFFCCF8093CE0008951F92E7
:101290000F920FB60F9211242F933F934F935F93AA
:1012A0008F939F93EF93FF938091BB0190E0AC01EC
:1012B0004F5F5F4F2091BA01241741F03091CE006B
:1012C000FC01E454FE4F30834093BB013091BB01DD
:1012D000822F90E0432F50E0841B950B321708F0CB
:1012E000939503970CF45D9AFF91EF919F918F91E5
:1012F0005F914F913F912F910F900FBE0F901F90D4
:1013000018958091D602089508958091D602089587
:101310000895089508950895CF93DF938D3C910526
:10132000B9F1B8F4853B9105A9F148F4833B9105E7
:10133000D1F1843B9105D1F5D0E0C0E23BC0873BC1
:10134000910571F150F18C3C910581F5D0E0C8E038
:1013500031C08A3E9105C1F040F4823E9105B1F062
:10136000893E910519F5D0E124C0813222E092072F
:1013700049F0833222E09207D9F08A389140B1F4E3
:10138000D2E017C0D4E015C0D0E213C0D0E411C041
:10139000D0E80FC0D0E0C1E00DC0D0E0C2E00AC08C
:1013A000D0E0C4E007C0D0E0C0E104C0D0E001C09C
:1013B000D1E0C0E08DEF0E94400983E00E94400927
:1013C00083E00E9440098D2F0E9440098C2FDF91FD
:1013D000CF910C944009CF93DF93EC018DEF0E94E5
:1013E000400985E00E94400982E00E94400988810E
:1013F0000E94400989810E9440098A810E94400917
:101400008B81DF91CF910C944009CF93DF93EC0156
:101410008DEF0E94400989E00E94400981E00E940E
:10142000400988810E94400980E00E9440098A8129
:101430000E9440098B810E9440098C810E944009D2
:101440008D810E9440098E810E9440098F81DF9129
:10145000CF910C9440090C941D09EF92FF920F93C9
:101460001F93CF938C010E94DB257C01C0E0C70154
:101470000E94F3258017910798F40E941D099C0192
:101480002F3F8FEF380751F02D3041F02A3041F0D7
:10149000EC2FF0E0E254FD4F2083CF5FC73138F3EB
:1014A000EC2FF0E0E254FD4F10828EEB92E0CF91F2
:1014B0001F910F91FF90EF9008950C94400981B314
:1014C000881F8827881F0895879A8F9A089585B75F
:1014D000806885BF85B7806885BF0E94640A86984A
:1014E0008E9A81988998559A5D980C940409879AE8
:1014F0008F9808958FB18695817008958FB186FB7E
:10150000882780F908958093D6020895CF93DF93BA
:10151000FC018491EF012196882321F00E9440096B
:10152000FE01F7CFDF91CF910895CF93DF93C2EB08
:10153000D1E00E941D098F3F2FEF920759F09F9332
:101540008F93DF93CF930E94D8070F900F900F9047
:101550000F90EFCFDF91CF9108950E94860A2FEF71
:1015600089E698E1215080409040E1F700C00000FA
:1015700084E690E00E942D0A8093BC029093BD0205
:101580009F938F9385EB91E09F938F930E94D80751
:101590000E94950A0F900F900F900F908091BC02BF
:1015A0009091BD0208950E946C189093150180934C
:1015B00014010E94381E80E091E00E9467180E948A
:1015C000770A0E947E0A8111FCCF8DE392E00E948F
:1015D0003F072FEF85EB95E3215080409040E1F7E6
:1015E00000C0000089E392E00E94AD0AEFEFFBE447
:1015F0002DE1E150F0402040E1F700C000000E94E2
:10160000950A85E392E00E94AD0AFC01808186374D
:1016100021F081E392E00C94AD0A089588E192E014
:101620000E943F0782E192E00E94AD0A0E94640A94
:101630000E94381E80911401909115010C94671836
:101640000E94C80F809121018093C80308958F9252
:101650009F92AF92BF92CF92DF92EF92FF920F9341
:101660001F93CF93DF9392E0B92E03E614E029E6AF
:10167000E22E24E0F22EAA24A39433E0932E41E537
:10168000C42E44E0D42E0E942B0AEC01019609F4EA
:1016900041C08091D9028130F9F028F0823009F1FF
:1016A000833021F134C0CE3FD10519F4A092D90284
:1016B000EACFC038D10528F4DF93CF93FF92EF92A1
:1016C00004C0DF93CF931F930F930E94D8070F900E
:1016D0000F900F900F90D7CF2297C9F4B092D902F4
:1016E000D2CF2197A1F49092D902CDCF8091B703A8
:1016F00080FF0AC0DF93CF93DF92CF920E94D8077A
:101700000F900F900F900F908C2F0E94830A1092D1
:10171000D902B9CF8091DB02811127C08091DA0212
:10172000811114C00E947A0A811110C00E946C18A5
:101730008A509140D1F00E94381E809121018093FF
:10174000C803109221018AE091E00DC00E946C183C
:101750008651914051F00E94381E8091C8038093B9
:10176000210186E191E00E9467188091D702909153
:10177000D8020E94F325893E23E0920708F461C055
:1017800028EE33E0B9010E94A02E629FC001639F42
:10179000900D729F900D11242091D7023091D802A4
:1017A000820F931F9093D8028093D7020E946610F5
:1017B000833011F481E001C080E00E94B70F0E94E5
:1017C000E72528EE33E040E050E00E94C82E4901B2
:1017D0005A018CE3C82ED12CE12CF12CCA01B9019D
:1017E000A70196010E94C82E672B682B692B49F52B
:1017F0000E942F102091B70320FF23C09F938F9347
:101800001F921F92C501B40120E13EE040E050E08C
:101810000E94C82EC22FA70196010E94C82E3F9396
:101820002F931F92CF938CE394E09F938F930E940A
:10183000D8078DB79EB70A960FB6F8949EBF0FBE15
:101840008DBF0E947A0A811107C00E947E0A8823F8
:1018500019F06E9A769802C06E9A769ADF91CF91BF
:101860001F910F91FF90EF90DF90CF90BF90AF90BE
:101870009F908F9008958F929F92AF92BF92CF9238
:10188000DF92EF92FF921F93CF93DF9300D000D0AF
:10189000CDB7DEB7833109F492C008F061C08B3058
:1018A00009F46CC008F055C0853009F003C20E94ED
:1018B000E72528EE33E040E050E00E94C82E4901C1
:1018C0005A010E942F109F938F938BE892E09F9371
:1018D0008F930E94D807C501B40120E13EE040E0AB
:1018E00050E00E94C82E5F934F933F932F9325E8BB
:1018F00032E03F932F9369837A838B839C830E948A
:10190000D8078CE3C82ED12CE12CF12C69817A8187
:101910008B819C81A70196010E94C82E5F934F93F3
:101920003F932F938FE792E09F938F930E94D80766
:10193000C501B401A70196010E94C82E9F938F9301
:101940007F936F9389E792E09F938F930E94D807CC
:101950004AC18C3009F441C0813109F4A4C1AAC143
:10196000883361F020F4883109F443C1A3C187347E
:1019700009F46AC18C3409F453C19CC188E194E034
:101980000E943F0783E094E00E943F0789EE93E0C6
:101990000E943F0782EC93E00E943F0787EA93E0B2
:1019A0000E943F0785E993E00E943F071091DB0208
:1019B000111111C085E793E00E943F077FC10E948B
:1019C000D30A8DE592E00E94AD0A87E592E00E947D
:1019D000AD0A0E940E0B11E071C18CE593E00E94EC
:1019E0003F070E946C188A50914019F080E391E003
:1019F00002C08AE291E09F938F938EE493E09F93DD
:101A00008F930E94D8078091DA021F928F938FE301
:101A100093E09F938F930E94D8070E947A0A0FB693
:101A2000F894DEBF0FBECDBF811107C00E947E0AB1
:101A3000811106C089E391E005C085E391E002C011
:101A40008CE391E09F938F9385E393E09F938F9333
:101A50000E94D8070E945F0A1F928F938AE193E049
:101A60009F938F930E94D8078091DB021F928F93E0
:101A700089E093E09F938F930E94D8078091CD03D4
:101A80000FB6F894DEBF0FBECDBF8823B9F08091AA
:101A9000CD038130B1F08091CD038230A9F08091E7
:101AA000CD038330A1F08091CD03843099F08091F3
:101AB000CD03853091F081E791E011C089E491E098
:101AC0000EC081E491E00BC084E591E008C08CE594
:101AD00091E005C086E691E002C083E791E09F9324
:101AE0008F938AEF92E09F938F930E94D80780EFA5
:101AF00092E09F938F930E94D8070E9466100F90E8
:101B00000F900F900F900F900F90813059F038F098
:101B1000823059F0833061F48AED92E00BC08BEE95
:101B200092E008C085EE92E005C08EED92E002C022
:101B300088ED92E09F938F930E94D8070F900F90AB
:101B400086ED92E09F938F930E94D8078091CB03FC
:101B50001F928F938DEB92E09F938F930E94D807F3
:101B60008091D90081701F928F9383EB92E09F93B5
:101B70008F930E94D8070E94E72528EE33E040E0CB
:101B800050E00E94C82E69017A019CE3892E912CB5
:101B9000A12CB12CCA01B901A50194010E94C82E43
:101BA0007F936F93C701B60120E13EE040E050E033
:101BB0000E94C82E122FA50194010E94C82E3F93A7
:101BC0002F931F921F93C701B60120E831E541E032
:101BD00050E00E94C82E3F932F9386E992E09F9396
:101BE0008F930E94D8070FB6F894DEBF0FBECDBF0B
:101BF000F2CE8091DB02811160C01091DA021123D4
:101C000039F08EE692E00E943F071092DA0256C049
:101C100084E692E00E943F0781E08093DA02DBCE07
:101C20000E945F0A182F882341F00E94D30A81E0A6
:101C30008093C7038093DB0241C00E940E0B109279
:101C4000C7031092DB02C7CE8091DB02811102C074
:101C50000E94D30A8BE092E00E94AD0A80E092E0FD
:101C60000E94AD0A8CEE91E00E94AD0A85EE91E0F3
:101C70000E94AD0A8BED91E00E94AD0A84ED91E0E7
:101C80000E94AD0A8AEC91E00E94AD0A80EC91E0DE
:101C90000E94AD0A8AEB91E00E94AD0A8091DB02BE
:101CA000811199CE96CE0E946C1811E08651914018
:101CB00029F403C01091DB0201C010E0812F0F90C6
:101CC0000F900F900F90DF91CF911F91FF90EF90A9
:101CD000DF90CF90BF90AF909F908F900895CF935B
:101CE000C82F0E949D24827291E009F490E04C2F4D
:101CF00050E0FA013497E934F10508F0D0C0EA5A0F
:101D0000FF4F0C94EA2E8BE12DC19111CCC081E6DE
:101D100029C19111CAC082E625C19111C8C083E6CC
:101D200021C19111C6C084E61DC19111C4C085E6D0
:101D300019C19111C2C086E615C19111C0C087E6D4
:101D400011C19111BEC088E60DC19111BCC089E6D8
:101D500009C19111BAC08AE605C19111B8C08BE6DC
:101D600001C19111B6C08CE6FDC09111B4C08DE6E1
:101D7000F9C09111B2C08EE6F5C09111B0C08FE6E6
:101D8000F1C09111AEC080E7EDC09111ACC081E708
:101D9000E9C09111AAC082E7E5C09111A8C083E70C
:101DA000E1C09111A6C084E7DDC09111A4C085E710
:101DB000D9C09111A2C086E7D5C09111A0C087E714
:101DC000D1C091119EC088E7CDC091119CC089E718
:101DD000C9C091119AC08AE7C5C0911198C081E32A
:101DE000C1C0911196C082E3BDC0911194C083E33C
:101DF000B9C0911192C084E3B5C0911190C085E340
:101E0000B1C091118EC086E3ADC091118CC087E343
:101E1000A9C091118AC088E3A5C0911188C089E347
:101E2000A1C0911186C080E39DC088E09BC089E07D
:101E300099C080E297C091117EC08DE293C091114C
:101E40007CC08DE38FC091117AC08BE58BC091115E
:101E500078C08DE587C0992309F475C08CE782C0EE
:101E6000992309F472C08CE77DC0911170C08BE397
:101E700079C091116EC087E275C091116CC080E687
:101E800071C091116AC08CE26DC0911168C08EE280
:101E900069C0911166C08FE265C080E063C080E2D6
:101EA00061C08AE05FC081E45DC082E45BC083E41E
:101EB00059C084E457C085E455C086E453C087E424
:101EC00051C088E44FC089E44DC08AE44BC08BE424
:101ED00049C08CE447C08DE445C08EE443C08FE424
:101EE00041C080E53FC081E53DC082E53BC083E560
:101EF00039C084E537C085E535C086E533C087E560
:101F000031C088E52FC089E52DC08AE52BC081E26C
:101F100029C080E427C083E225C084E223C085E293
:101F200021C08EE51FC086E21DC08AE21BC088E288
:101F300019C089E217C08FE515C08BE213C08BE78B
:101F400011C08DE70FC08CE50DC08CE50BC08AE396
:101F500009C082E207C08EE705C08CE303C08EE3B0
:101F600001C08FE30E945D0A81E0CF910895833024
:101F700019F4859A7D9A0895813011F4859A06C0E6
:101F8000823019F4859A8D9A089585988D980895D0
:101F900081E00E94B70F2FEF81EE94E02150804046
:101FA0009040E1F700C0000082E00E94B70F2FEFE1
:101FB00081EE94E0215080409040E1F700C00000A5
:101FC00081E00E94B70F2FEF81EE94E02150804016
:101FD0009040E1F700C0000082E00E94B70F2FEFB1
:101FE00081EE94E0215080409040E1F700C0000075
:101FF00080E00E94B70F80EC80937C0087E08093A4
:102000007A0081E980937E0081E080937F008BE3FA
:1020100080937D00849A8C9808958091D90080FFE8
:102020001CC090B331B385988D9AEFE9FFE03197EA
:10203000F1F700C000008FB185FB882780F920B33D
:1020400090722F7D292B20BB91B3232F20729F7D6F
:10205000922B91BB91E08927089580E00895CF935A
:10206000DF9300D0CDB7DEB7849A8C9A80917A0046
:10207000806880937A008FE99FE00197F1F700C0B4
:10208000000080917A00806480937A0080917A00C9
:1020900086FDFCCF80917800909179009A838983A6
:1020A00080917A008F7780937A00849A8C98298126
:1020B0003A8145E0429FC001439F900D1124805515
:1020C00091090F900F90DF91CF9108958091D900E1
:1020D00080FD0C940D100E942F108C3A2DE0920779
:1020E00020F481E08093DC0205C085379E4010F02B
:1020F0001092DC028091DC02811102C082E008951E
:1021000083E00895CF93C82F0E94FC068C2F0E9475
:10211000041180E0CF91089584B7877F84BF0FB604
:10212000F894A89580916000886180936000109277
:1021300060000FBE90E080E80FB6F89480936100D5
:10214000909361000FBE0E9485150E94E215809158
:10215000E20084608093E20082E890E10E943925E9
:10216000509A589A5198599A78948FEF9091CD033C
:102170008150943041F0EFE7FEE33197F1F700C072
:1021800000008111F3CF8CE894E00E943F070E9489
:10219000670A0E94200B80E894E00E943F070E949B
:1021A0002D1980E794E00E943F070E947A0A882355
:1021B00019F18091CD038530F9F48CE694E00E940A
:1021C0003F070E94FB080E9468250E9468250E9424
:1021D00068250E9468250E9468250E9468250E9443
:1021E00068258091CB03882301F30E9491258823E1
:1021F000E1F20E94DA13D9CF0E9431190E94270B15
:10220000D4CF8091010308959FB7F8941092E00213
:102210009FBF9091CD03943009F057C09091E90091
:102220009F703091EC00232F217030FD20E8922B1D
:1022300024E02093E9002091EB0020FF43C020918F
:10224000EE0027FF3FC02091DD02222321F02091E4
:10225000E80025FF37C01092DD0226E03091E8004B
:1022600035FD15C03091CD03343061F53091EB0070
:1022700035FD28C0215021F481E08093DD0222C089
:10228000EFE9FFE03197F1F700C00000E7CF80935E
:10229000F1008091E80085FD0AC08091E80080FF90
:1022A000FCCF8091E8008E778093E80006C08FB75E
:1022B000F89421E02093E0028FBF9F709093E90093
:1022C00080E008959F709093E9008FEF0895CF9379
:1022D000DF9300D01F92CDB7DEB79C018091CD0374
:1022E000843019F593E099833B832A839093E90026
:1022F0008FEF9091E800815095FD06C095ED9A957D
:10230000F1F700008111F5CF8091E80085FF0DC045
:1023100040E050E063E070E0CE0101960E94F013CF
:102320008091E8008E778093E8000F900F900F90D7
:10233000DF91CF910895CF93DF9300D01F92CDB757
:10234000DEB72091CD03243021F522E029839B8341
:102350008A8383E08093E9008FEF9091E8008150B9
:1023600095FD06C095ED9A95F1F700008111F5CF26
:102370008091E80085FF0DC040E050E063E070E030
:10238000CE0101960E94F0138091E8008E77809331
:10239000E8000F900F900F90DF91CF91089520915A
:1023A000CD032430F1F422E02093E9002FEF3091A7
:1023B000E800215035FD06C035ED3A95F1F70000F3
:1023C0002111F5CF2091E80025FF0BC040E050E03F
:1023D00065E070E00E94F0138091E8008E778093B2
:1023E000E8000895CF93DF932091CD03243009F0C6
:1023F00048C0EC01809120018823E1F08091210107
:102400008823C1F085E08093E9008FEF9091E80088
:10241000815095FD06C09AE29A95F1F700C08111AE
:10242000F5CF8091E80085FF2CC040E050E060E2ED
:1024300070E017C081E08093E9008FEF9091E80091
:10244000815095FD06C095ED9A95F1F70000811138
:10245000F5CF8091E80085FF14C040E050E068E0CF
:1024600070E0CE010E94F0138091E8008E77809397
:10247000E80080E2FE01A1EEB2E001900D928A95A3
:10248000E1F7DF91CF9108958BE994E00E943F0737
:102490008091CC03811109C00E9485150E94E2152C
:1024A0008091E20084608093E200089587E994E0DF
:1024B0000E943F071092CC03089508952091DE02F8
:1024C0002F5F822F62E30E94942E992319F02093AC
:1024D000DE0208951092DE028091E002882371F1FD
:1024E0008091CD03843041F58091E9008F70209177
:1024F000EC00922F917020FD90E8892B94E090934E
:10250000E9009091EB0090FF14C09091EE0097FFCE
:1025100010C09091E80095FF03C01092F100F9CF30
:102520009091E80090FF05C09091E8009E7790930D
:10253000E8008F708093E9001092E002089542E075
:1025400061EC81E00E94FF1442E061EC82E00E94B5
:10255000FF1442E061EC83E00E94FF1442E261EC70
:1025600084E00E94FF1442E261EC85E00C94FF14C9
:102570008091CF03833009F455C030F4813071F07D
:10258000823009F48EC008958A3009F47AC08B3005
:1025900009F460C0893009F09CC020C08091CE034E
:1025A000813A09F096C08091E800877F8093E80027
:1025B0008091D2039091D303892B21F460E281EEC4
:1025C00092E003C060E080E090E070E00E943B1485
:1025D0008091E8008B778093E80008958091CE0386
:1025E000813209F076C08091D2039091D303009795
:1025F00019F0049709F06DC08091E800877F8093FF
:10260000E8008091E80082FD05C08091CD03811132
:10261000F8CF5FC08091F100809301038091E800C2
:102620008B7753C08091CE03813A09F052C08091DC
:10263000D2039091D303892B09F04BC08091E8001D
:10264000877F8093E8008091E80080FFFCCF809135
:10265000200136C08091CE038132D9F58091D2031A
:102660009091D303892BA9F58091E800877F80930F
:10267000E8000E9434158091D003809320010C94CF
:10268000381E8091CE03813221F58091E800877F4A
:102690008093E8000E9434158091D1038093020357
:1026A00008958091CE03813AA1F48091E800877F5C
:1026B0008093E8008091E80080FFFCCF80910203C6
:1026C0008093F1008091E8008E778093E8000C946D
:1026D00034150895809101038093DF021092010365
:1026E00080E00E94FD080E94D6190C94381E0C94BC
:1026F0006A130E94A5258091DF028093010308954B
:102700000C947913292F332723303105C9F064F451
:102710002130310581F02230310509F043C08DE8C8
:1027200090E027EC34E042C021323105F1F0223252
:10273000310541F137C082E190E024E535E036C053
:1027400099278130910541F08230910541F0892B24
:1027500049F5E3ECF4E005C0E3EBF4E002C0EFE997
:10276000F4E0849190E09F0121C06530D8F4E62F19
:10277000F0E0EE0FFF1FE457FE4F2081318189E02A
:1027800090E014C0653070F470E0FB01EE0FFF1FA5
:10279000EE57FE4F20813181FB01E358FE4F8081CF
:1027A00090E004C080E090E020E030E0FA01318366
:1027B0002083089580E189BD82E189BD09B400FECE
:1027C000FDCF8091D8008F7D8093D8008091E0006C
:1027D00082608093E0008091E00081FDFCCF08954D
:1027E000CF92DF92EF92FF920F931F93CF93DF93DD
:1027F000EC018B016A010E945315811133C0C11491
:10280000D10439F0F60180819181081B190BC80FA2
:10281000D91FE12CF12C0115110519F18091E80067
:1028200085FD16C08091E8008E778093E800C11482
:10283000D10449F0F60180819181E80EF91EF18200
:10284000E08285E00FC00E945315882321F30AC05F
:1028500089918093F10001501109FFEFEF1AFF0AEF
:10286000DACF80E0DF91CF911F910F91FF90EF9031
:10287000DF90CF9008952091D4033091D50326178F
:10288000370748F06115710539F42091E8002E777B
:102890002093E80001C0B90140E061157105A9F17C
:1028A0002091CD03222309F443C0253009F442C00E
:1028B0002091E80023FD40C02091E80022FD32C0B5
:1028C0002091E80020FFE9CF4091F3002091F20031
:1028D00030E0342BFC01CF016115710559F028302F
:1028E000310540F481918093F100615071092F5FAF
:1028F0003F4FF1CF41E02830310509F040E0209111
:10290000E8002E772093E800C8CF4111C9CF0AC054
:102910008091CD03882361F0853061F08091E800DB
:1029200083FD0AC08091E80082FFF2CF80E0089525
:1029300082E0089583E0089581E008952091D40312
:102940003091D5032617370748F06115710539F422
:102950002091E8002E772093E80001C0B901FC0126
:1029600020E06115710591F18091CD03882309F470
:1029700040C0853009F43FC08091E80083FD3DC030
:102980008091E80082FD2FC08091E80080FFE9CFB0
:102990002091F3008091F20090E0922B6115710577
:1029A00059F08830910540F424912093F10031963C
:1029B000615071090196F2CF21E0089709F020E0FB
:1029C0008091E8008E778093E800CBCF2111CCCFA7
:1029D0000AC08091CD03882361F0853061F0809139
:1029E000E80083FD0AC08091E80082FFF2CF80E01A
:1029F000089582E0089583E0089581E00895982F76
:102A0000973058F59093E900981739F07091EC00E1
:102A10002091ED005091F00003C0242F762F50E05C
:102A200021FF19C03091EB003E7F3093EB003091D5
:102A3000ED003D7F3093ED003091EB00316030933D
:102A4000EB007093EC002093ED005093F000209188
:102A5000EE0027FF07C09F5FD3CF8F708093E90000
:102A600081E0089580E008958091CE0387FF11C032
:102A70008091E80082FD05C08091CD038111F8CFDF
:102A800011C08091E8008B770BC08091CD03882323
:102A900049F08091E80080FFF8CF8091E8008E77C0
:102AA0008093E80008952091E4003091E50095E6D8
:102AB0004091EC00842F817040FF22C08091E8009B
:102AC00080FD1CC08091CD03882391F0853091F06A
:102AD0008091EB0085FD10C04091E4005091E5002D
:102AE0004217530729F39A01915011F784E0089592
:102AF00082E0089583E0089581E0089580E00895DC
:102B00004091E80042FFDECF08950E94F3150E9435
:102B1000FB15E0EEF0E0808181608083E8EDF0E07D
:102B200080818F77808319BCA7EDB0E08C918E7F78
:102B30008C9380818F7E80831092CC0308950F93B5
:102B40001F93CF93DF930E94F3150E94FB15C8EDEE
:102B5000D0E088818F7788838881806888838881A6
:102B60008F7D888319BC1092CD031092C9031092F7
:102B7000CB031092CA0300EE10E0F80180818B7F36
:102B8000808388818160888342E060E080E00E94E9
:102B9000FF14E1EEF0E080818E7F8083E2EEF0E0D2
:102BA000808181608083808188608083F80180815A
:102BB0008E7F8083888180618883DF91CF911F9190
:102BC0000F910895E8EDF0E080818F7E8083E7ED3E
:102BD000F0E080818160808384E082BF81E0809327
:102BE000CC030C949F15E8EDF0E080818E7F80830C
:102BF0001092E20008951092DA001092E100089518
:102C00001F920F920FB60F9211242F933F934F9361
:102C10005F936F937F938F939F93AF93BF93EF9344
:102C2000FF938091E10082FF0BC08091E20082FF60
:102C300007C08091E1008B7F8093E1000E945E12CB
:102C40008091DA0080FF1FC08091D80080FF1BC0F8
:102C50008091DA008E7F8093DA008091D90080FF26
:102C60000DC080E189BD82E189BD09B400FEFDCFC0
:102C700081E08093CD030E94441205C019BC1092DC
:102C8000CD030E9456128091E10080FF19C080910F
:102C9000E20080FF15C08091E2008E7F8093E20009
:102CA0008091E20080618093E2008091D800806290
:102CB0008093D80019BC85E08093CD030E947713E0
:102CC0008091E10084FF30C08091E20084FF2CC03D
:102CD00080E189BD82E189BD09B400FEFDCF80910C
:102CE000D8008F7D8093D8008091E1008F7E809303
:102CF000E1008091E2008F7E8093E2008091E2000B
:102D000081608093E2008091C903882311F084E000
:102D100007C08091E30087FD02C081E001C083E02D
:102D20008093CD030E9480138091E10083FF29C02E
:102D30008091E20083FF25C08091E100877F80932E
:102D4000E10082E08093CD031092C9038091E100FD
:102D50008E7F8093E1008091E2008E7F8093E2007D
:102D60008091E20080618093E20042E060E080E0D8
:102D70000E94FF148091F00088608093F0000E9410
:102D80005D12FF91EF91BF91AF919F918F917F91D4
:102D90006F915F914F913F912F910F900FBE0F90C8
:102DA0001F9018951F920F920FB60F9211242F9318
:102DB0003F934F935F936F937F938F939F93AF93C3
:102DC000BF93CF93DF93EF93FF93C091E900CF7050
:102DD0008091EC00D82FD17080FDD0E81092E900EE
:102DE0008091F000877F8093F00078940E941617FE
:102DF0001092E9008091F00088608093F000CD2B64
:102E0000CF70C093E900FF91EF91DF91CF91BF9117
:102E1000AF919F918F917F916F915F914F913F9172
:102E20002F910F900FBE0F901F9018951F93CF9367
:102E3000DF93CDB7DEB7AA970FB6F894DEBF0FBE0B
:102E4000CDBFEEECF3E088E08E0F9091F10091930E
:102E50008E13FBCF0E94B8128091E80083FF1FC140
:102E60008091CE039091CF03492F50E04A30510515
:102E700008F015C1FA01E156FF4F0C94EA2E803894
:102E800081F0823809F00BC18091D2038F7080935A
:102E9000E9008091EB0085FB882780F91092E9001A
:102EA00006C08091CA039091CB03911182609091EA
:102EB000E800977F9093E8008093F1001092F10072
:102EC000C8C0282F2D7F09F0EAC0882319F082306E
:102ED00061F0E5C08091D003813009F0E0C093300B
:102EE00009F080E08093CB032BC08091D003811147
:102EF00027C08091D2038F7009F4D1C08093E9007C
:102F00002091EB0020FF1CC0933021F48091EB0056
:102F1000806214C09091EB0090619093EB0021E0EF
:102F200030E0A90102C0440F551F8A95E2F7409393
:102F3000EA001092EA008091EB0088608093EB0039
:102F40001092E9008091E800877F86C08111A7C0B8
:102F50001091D0031F778091E3008078812B8093BC
:102F6000E3008091E800877F8093E8000E94341599
:102F70008091E80080FFFCCF8091E300806880931F
:102F8000E300111102C082E001C083E08093CD0311
:102F900086C08058823008F082C08091D003909122
:102FA000D1038C3D53E0950779F583E08A838AE26B
:102FB00089834FB7F894DE01139620E03EE051E29A
:102FC000E32FF0E050935700E49120FF03C0E29517
:102FD000EF703F5FEF708E2F90E0EA3010F0C796F1
:102FE00001C0C0968D939D932F5F243149F74FBF49
:102FF0008091E800877F8093E8006AE270E0CE016C
:1030000001960E943B1414C0AE014F5F5F4F609168
:10301000D2030E948213BC01892B09F440C0909115
:10302000E800977F9093E80089819A810E949E141E
:103030008091E8008B778093E80031C0803879F583
:103040008091E800877F8093E8008091C903809396
:10305000F1008091E8008E778093E8000E9434159B
:103060001EC081111CC09091D0039230C0F4809199
:10307000E800877F8093E8009093C9030E9434158D
:103080008091C903811106C08091E30087FD02C0D1
:1030900081E001C084E08093CD030E949F12809163
:1030A000E80083FF0AC08091E800877F8093E800F2
:1030B0008091EB0080628093EB00AA960FB6F894A3
:1030C000DEBF0FBECDBFDF91CF911F9108959093CA
:1030D00008038093070308958091070390910803E4
:1030E0000895E0910703F0910803309721F00190D3
:1030F000F081E02D099480E00895EF92FF920F9304
:103100001F93CF93DF93E0910703F091080330976B
:10311000B1F18C010280F381E02D09958091B70314
:1031200082FF2DC080FF04C08AEA96E00E943F071C
:10313000E80110E284EAE82E86E0F82E8091B703D9
:1031400080FF0BC088811F928F93FF92EF920E94A5
:10315000D8070F900F900F900F90115021961111DA
:10316000EDCF8091B70380FF0AC082EA96E0DF913D
:10317000CF911F910F91FF90EF900C943F07DF913B
:10318000CF911F910F91FF90EF900895E091070369
:10319000F0910803309721F00480F581E02D099427
:1031A0000895CF93DF93EC0180910503909106037E
:1031B000C817D90709F1D0930603C0930503E0911E
:1031C0000703F09108033097B9F00680F781E02DEE
:1031D000CE0109958091B70382FF0EC080FF0CC01D
:1031E000DF93CF9384E996E09F938F930E94D80753
:1031F0000F900F900F900F90DF91CF910895CF9384
:10320000DF93EC018091030390910403C817D90761
:1032100009F1D0930403C0930303E0910703F091F5
:1032200008033097B9F00084F185E02DCE010995AF
:103230008091B70382FF0EC080FF0CC0DF93CF9355
:1032400084E896E09F938F930E94D8070F900F9089
:103250000F900F90DF91CF9108950E94D2250C948A
:10326000F407BF92CF92DF92EF92FF920F931F93DA
:10327000CF93DF9300D000D01F92CDB7DEB70E946E
:103280001F080AE013E0F12C8F2D0E94F008B82EE1
:10329000F801C080C82639F4F3940F5F1F4FF8E09F
:1032A000FF12F2CF30C08091B70381FD0E94D71981
:1032B000D12CEE24E3948E2D8C21F9F0D982FA8260
:1032C00081E09E2D9B2109F480E08B830E94DB2509
:1032D0008160782F9D838C8349815A816B818D8198
:1032E0000E940B1A49815A816B817C818D810E94D9
:1032F0005525F80190819E259083D394EE0CF8E03B
:10330000DF12D9CFC9CF8FEF89838A831B820E94B6
:10331000DB258160782F9D838C8349815A816B8165
:103320008D810E940B1A0E9454250E94C82810917A
:1033300009030E947118181741F10E9471188093B7
:1033400009039091B70392FF0EC090FF0CC01F922B
:103350008F9385EB96E09F938F930E94D8070F90F1
:103360000F900F900F90809109030F900F900F9086
:103370000F900F90DF91CF911F910F91FF90EF90E1
:10338000DF90CF90BF900C9466250F900F900F9018
:103390000F900F90DF91CF911F910F91FF90EF90C1
:1033A000DF90CF90BF9008950C94FD080895EF92A0
:1033B000FF920F931F93CF93DF938EEC96E00E94C2
:1033C0003F07C0E0D0E08FE2E82E81E0F82E00EC6D
:1033D00016E08C2F0E94F0080E943E25FF92EF928B
:1033E0001F928F93DF93CF931F930F930E94D80761
:1033F00021968DB79EB708960FB6F8949EBF0FBE64
:103400008DBFC830D10529F7DF91CF911F910F9162
:10341000FF90EF900895CF93DF93CDB7DEB72B9752
:103420000FB6F894DEBF0FBECDBF942F4F83252F6C
:10343000588769877A878B874A855B85452B21F07A
:103440002F3F09F59F3FF9F4DE01119686E0FD015B
:1034500011928A95E9F785E0FE01379601900D9269
:103460008A95E1F749815A816B817C818D819E81AA
:103470000E941D212B960FB6F894DEBF0FBECDBF64
:10348000DF91CF9108954F81588569857A858B8525
:103490000E945525D9CFCF93882309F465C0C82F42
:1034A0008CEF8C0F813A20F080E58C0F8E3248F43F
:1034B0008C2F0E940E2C811157C08C2F0E94F52357
:1034C0000CC080E28C0F883058F4C77081E001C0D6
:1034D000880FCA95EAF70E94A024CF910C94E424A7
:1034E0008BE58C0F833078F4C53A29F0C63A31F079
:1034F00083E890E005C081E890E002C082E890E0B7
:10350000CF910C94D11888E58C0F853168F5C83AB5
:1035100089F0C93A91F0CA3A99F0CB3AA1F0CC3A85
:10352000A9F0CD3AB1F0CE3AB9F0CF3AC1F080E08F
:1035300090E017C082EE90E014C089EE90E011C0D8
:103540008AEE90E00EC085EB90E00BC086EB90E039
:1035500008C083EB90E005C084EB90E002C087EBED
:1035600090E0CF910C94FF18CF910895882349F1F2
:103570009CEF980F913A20F090E5980F9E3218F446
:103580000E9448240DC090E2980F983058F487703C
:1035900091E001C0990F8A95EAF7892F0E94A6242D
:1035A0000C94E4249BE5980F933020F480E090E0A5
:1035B0000C94D118885A853120F480E090E00C9466
:1035C000FF180895882321F00E94A0240C94E4247D
:1035D0000895882321F00E94A6240C94E4240895E1
:1035E000BF92CF92DF92EF92FF920F931F93CF93F0
:1035F000DF9300D000D000D0CDB7DEB725E0FC01CE
:10360000DE01119601900D922A95E1F7FC014081AF
:103610005181028163817481258122952F7061150A
:10362000710509F403C35F3F19F44F3F09F4FEC26B
:103630006C01862F7D836C83602F782F8D812E8384
:103640000E947923182FB92E0E9478230E946822A5
:10365000EB2DE295EF70F0E0E755FF4F2E810C94D3
:10366000EA2E8B2D807F9B2D9F70F92E882319F0D9
:10367000F29490EFF922002349F0FF2009F483C26D
:103680008F2D0E94B3240E94E4247DC2812F0E94CA
:10369000B61AFF2009F4CAC28F2D0E94B9242696BB
:1036A0000FB6F894DEBF0FBECDBFDF91CF911F9153
:1036B0000F91FF90EF90DF90CF90BF900C94E42497
:1036C0008B2D807F9B2D9F70F92E803219F0F29404
:1036D00080EFF822112319F0113009F12AC00023DC
:1036E000B1F08F2D222351F1213041F526960FB6EE
:1036F000F894DEBF0FBECDBFDF91CF911F910F9128
:10370000FF90EF90DF90CF90BF900C94C3242223C2
:1037100019F0213009F48AC20E94CC242DC0002364
:10372000F1F0263008F082C20E949D248F2129F0FA
:1037300023C00023F9F0211116C08F2D26960FB655
:10374000F894DEBF0FBECDBFDF91CF911F910F91D7
:10375000FF90EF90DF90CF90BF900C94E21A25304D
:1037600008F064C209C0F601858180FF0CC28F7029
:103770008583E3CF21111CC28F2D83C12B2D26956C
:103780002695237030E02115310521F021303105D7
:10379000D1F04CC2002321F0812F9B2D937002C0E9
:1037A00080E090E026960FB6F894DEBF0FBECDBF46
:1037B000DF91CF911F910F91FF90EF90DF90CF900D
:1037C000BF900C94D118002321F0812F9B2D937072
:1037D00002C080E090E026960FB6F894DEBF0FBEE0
:1037E000CDBFDF91CF911F910F91FF90EF90DF90B0
:1037F000CF90BF900C94FF18812F002319F00E94E6
:103800004E2702C00E94B62726960FB6F894DEBF58
:103810000FBECDBFDF91CF911F910F91FF90EF9021
:10382000DF90CF90BF900C943B288B2D837009F0D4
:103830007BC00111FBC1812F829586958770880F0F
:10384000880F912F9F70C92ED12CE12CF12C082EBE
:1038500004C0CC0CDD1CEE1CFF1C0A94D2F714FF34
:1038600012C04FE050E060E070E004C0440F551F0C
:10387000661F771F8A95D2F7CB01BA0160957095C4
:103880008095909503C060E070E0CB012B2D2695CC
:1038900026952370422F50E042305105D9F0433035
:1038A000510569F16C297D298E299F2941305105E7
:1038B00051F126960FB6F894DEBF0FBECDBFDF9153
:1038C000CF911F910F91FF90EF90DF90CF90BF901D
:1038D0000C948D226C297D298E299F2926960FB65E
:1038E000F894DEBF0FBECDBFDF91CF911F910F9136
:1038F000FF90EF90DF90CF90BF900C94A7220E9492
:103900008D22C701B60126960FB6F894DEBF0FBE12
:10391000CDBFDF91CF911F910F91FF90EF90DF907E
:10392000CF90BF900C947322002319F08B2D8170DF
:1039300001C08695882309F479C1812F82958695E7
:103940008770880F880F912F9F70C92ED12CE12C82
:10395000F12C082E04C0CC0CDD1CEE1CFF1C0A94BC
:10396000D2F714FF12C04FE050E060E070E004C0F6
:10397000440F551F661F771F8A95D2F7CB01BA01F6
:10398000609570958095909503C060E070E0CB01E4
:103990002B2D269526952370422F50E0423051055D
:1039A000D9F04330510569F16C297D298E299F2971
:1039B0004130510551F126960FB6F894DEBF0FBE87
:1039C000CDBFDF91CF911F910F91FF90EF90DF90CE
:1039D000CF90BF900C9454236C297D298E299F2968
:1039E00026960FB6F894DEBF0FBECDBFDF91CF9104
:1039F0001F910F91FF90EF90DF90CF90BF900C94AC
:103A000066230E945423C701B60126960FB6F89488
:103A1000DEBF0FBECDBFDF91CF911F910F91FF9001
:103A2000EF90DF90CF90BF900C944223103FD1F1E4
:103A300028F480E4810F803250F0A0C0123F09F4D6
:103A400062C008F44BC0133F09F472C097C0F12F55
:103A5000F071FF2E8B2D8F71002351F00E94DB221D
:103A6000812FFF2019F08295807F68CE8F7066CEFF
:103A70000E94FC22812FFF2019F08295807F01C0D7
:103A80008F7026960FB6F894DEBF0FBECDBFDF91C4
:103A9000CF911F910F91FF90EF90DF90CF90BF904B
:103AA0000C94E91A0023B1F0253008F0BFC08B2D2B
:103AB0008F7126960FB6F894DEBF0FBECDBFDF9193
:103AC000CF911F910F91FF90EF90DF90CF90BF901B
:103AD0000C942123263008F0A9C0E9CF0023A9F0D7
:103AE0008B2D8F7126960FB6F894DEBF0FBECDBF1B
:103AF000DF91CF911F910F91FF90EF90DF90CF90CA
:103B0000BF900C94DB22002359F38B2D8F712696E6
:103B10000FB6F894DEBF0FBECDBFDF91CF911F91DE
:103B20000F91FF90EF90DF90CF90BF900C94FC220C
:103B3000002399F08B2D8F7126960FB6F894DEBF77
:103B40000FBECDBFDF91CF911F910F91FF90EF90EE
:103B5000DF90CF90BF900C94C62226960FB6F894B3
:103B6000DEBF0FBECDBFDF91CF911F910F91FF90B0
:103B7000EF90DF90CF90BF900C94C1220023A9F06A
:103B8000222309F4ADCF812F26960FB6F894DEBF1D
:103B90000FBECDBFDF91CF911F910F91FF90EF909E
:103BA000DF90CF90BF900C944B1A222309F4ADCF35
:103BB000812F26960FB6F894DEBF0FBECDBFDF91E2
:103BC000CF911F910F91FF90EF90DF90CF90BF901A
:103BD0000C94B61A4B2D4F70612FC6010E94C82657
:103BE00026960FB6F894DEBF0FBECDBFDF91CF9102
:103BF0001F910F91FF90EF90DF90CF90BF900C94AA
:103C0000C1214B2D4F70612FC60126960FB6F89437
:103C1000DEBF0FBECDBFDF91CF911F910F91FF90FF
:103C2000EF90DF90CF90BF900C94CB2626960FB6E6
:103C3000F894DEBF0FBECDBFDF91CF911F910F91E2
:103C4000FF90EF90DF90CF90BF9008950E94C02426
:103C50000E948F240E94E4240E946D290E943B2828
:103C600080E090E00E94D11880E090E00C94FF1872
:103C70000E94B0240C94261ECF93DF9300D000D076
:103C80001F92CDB7DEB7942F4983252F5A836B83BC
:103C90007C838D834C815D81452B39F12F3F11F45D
:103CA0009F3F19F149815A816B817C818D810E94EE
:103CB0007923292F22952F7030E02C30310504F51F
:103CC0002A3031055CF4225031092230310568F484
:103CD000853A80F4843090F4823080F0883E38F465
:103CE000803E60F48450813A48F080E014C0803F08
:103CF000E1F704C090E2980F983080F781E00BC0A4
:103D00002C30310521F493FB882780F904C02F3033
:103D10003105C9F3EACF0F900F900F900F900F90DD
:103D2000DF91CF910895CF93DF9300D000D01F9201
:103D3000CDB7DEB70F900F900F900F900F90DF91DF
:103D4000CF910895CF93DF9300D000D000D0CDB7AE
:103D5000DEB726960FB6F894DEBF0FBECDBFDF915B
:103D6000CF9108951F93CF93DF93C091120316E074
:103D700080911303C81799F0D0E01C9FF0011D9F9C
:103D8000F00D1124EC5EFC4F408151816281738102
:103D9000848195810E94A21E2196C770E9CFDF9190
:103DA000CF911F9108954091440350914503609134
:103DB00046037091470380914803909149030C9406
:103DC000A21E8091490382958F7009F054C08091A2
:103DD0004603882309F44FC080911203A091130376
:103DE000609144037091450340914703509148030B
:103DF000B6E08A1709F43FC090E041155105C1F1C2
:103E00007F3F11F46F3FA1F1B89FF001B99FF00D12
:103E10001124EC5EFC4F218172132AC020816213B1
:103E200027C02281211124C0238134812417350722
:103E300010F421503109241B350B2C323140C0F4D1
:103E4000209149032F7020612093490326E0289F89
:103E5000F001299FF00D1124E75EFC4F80818F70E7
:103E60008061808384E493E00E94F01A0C94B21E77
:103E700001968770BECF0895BF92CF92DF92EF92E6
:103E8000FF920F931F93CF93DF93CDB7DEB7619768
:103E90000FB6F894DEBF0FBECDBF7C0185E0F70101
:103EA000DE011D9601900D928A95E1F7D7014C91A4
:103EB00011965C9111971296DC90129713960D91C2
:103EC0001C911497309144036091450380914703FE
:103ED00090914803009709F47FC16F3F19F43F3F69
:103EE00009F47AC1B0904603BB2009F4CAC02091FE
:103EF00049030817190750F0F801E81BF90BCF0127
:103F0000CC24C3948C329140D0F009C08095909518
:103F1000800F911FCC24C3948C32914080F0C12C2F
:103F2000207F09F0CCC0702F198B088B6D2D8989EB
:103F30000E94931E84E493E00E94F01AB6C0822F80
:103F4000807F09F047C0651314C0341312C0D1102C
:103F500010C02F702061209349030E94D31E84E477
:103F600093E00E94F01A80914903D70115968C9333
:103F70002FC00115110519F15F3F11F44F3FF9F002
:103F8000CD2CD1101CC0809112032091130336E078
:103F9000821709F45CC090E0389FF001399FF00D62
:103FA0001124EC5EFC4F6181561306C060814613FC
:103FB00003C06281611103C001968770E9CFCD2CE7
:103FC000DD2009F429C18091490381608093490370
:103FD000C12C22C1651308C0341306C0D11004C01F
:103FE00080914903D701CCC04D875E87DF86702F53
:103FF000198B088B6D2D89890E943C1E8823E9F15D
:10400000DD20D9F120914903822F82958F7090E0B5
:10401000029774F0809144039091450398878F83B1
:1040200019861B870A872C87CE0107960E94F01AF3
:1040300086E0F701A4E4B3E001900D928A95E1F7E0
:104040000E94E11E0E94D31ECC24C394E5C0702FB1
:10405000198B088B60E089890E947923292F22958A
:104060002F7030E0223031050CF0CAC09F7009F08B
:10407000C4C0805E883008F4CFC0C7010E94F01A27
:10408000E3CF0817190708F456C0F801E81BF90B2D
:10409000CF018C32914008F456C0C12C702F198B7F
:1040A000088B6D2D89890E94931EE4E4F3E086E07D
:1040B000DF011D928A95E9F70E94D31EADC06513FA
:1040C00014C0341312C0D11010C080914903F701FD
:1040D0008583C7010E94F01A86E0E4E4F3E0DF0183
:1040E0001D928A95E9F7CB2C97C04D875E87DF86B6
:1040F000702F198B088B6D2D89890E943C1E882397
:1041000009F4BBCFDD2009F4B8CF20914903822FF9
:1041100082958F7090E002970CF48ACF80914403CF
:10412000909145039A8389831B821D830C832E8380
:10413000CE0101967BCF80959095800F911F8C3298
:10414000914008F0AACFCD2CDD2009F496CF65135D
:104150002EC034132CC02091490320FD1FC0822F94
:1041600082958F70D9F0D70115962C9315978F30C3
:1041700049F08F5F982F9295907F822F8F70892BB7
:1041800015968C93C7010E94F01A86E0F701A4E40B
:10419000B3E001900D928A95E1F78ECF86E0F701AA
:1041A000A4E4B3E001900D928A95E1F735C04D8704
:1041B0005E87DF86702F198B088B6D2D89890E9491
:1041C0003C1E811135CF8091490381608093490362
:1041D000C7010E94F01A20C0DD2009F44ECF4D87A0
:1041E0005E87DF86702F198B088B6D2D89890E9461
:1041F0003C1E882309F441CF1BCF81113ACF0CC05C
:10420000243031050CF039CF9F7009F432CFF7011B
:104210009581907F09F02DCF8C2D61960FB6F89483
:10422000DEBF0FBECDBFDF91CF911F910F91FF90E9
:10423000EF90DF90CF90BF9008951F93CF93DF93BF
:10424000CDB7DEB72C970FB6F894DEBF0FBECDBF4B
:104250004F83588769877A878B879C87CE0107961B
:104260000E943C1F882369F08F8198852A853B85B1
:10427000232BF1F19F3F09F063C08F3F09F060C02D
:1042800037C086E0FE013796DE01119601900D924F
:104290008A95E1F76F817885EA85FB85309741F152
:1042A0007F3F11F46F3F21F12091130330E0C901EA
:1042B0000196877099274091120350E08417950763
:1042C00009F447C069837A83FD83EC8396E0929F6B
:1042D000D001939FB00D1124AC5EBC4FFE0131960E
:1042E00001900D929A95E1F7809313030E94B21EFC
:1042F00016E080911203909113038917C1F1189F62
:10430000C00111248C5E9C4F0E943C1F882379F1D0
:10431000E09112031E9FF0011124EC5EFC4F4081DE
:10432000518162817381848195810E94A21E809156
:10433000120390E001968770992780931203D9CFDA
:104340004F81588569857A858B859C850E94A21E40
:10435000CFCF0E94381E1092130310921203E4E490
:10436000F3E086E0DF011D928A95E9F7C1CF2C9634
:104370000FB6F894DEBF0FBECDBFDF91CF911F9176
:104380000895DF92EF92FF920F931F93CF93DF93E5
:10439000FC01892B09F48AC0E12CF12CDD24D39493
:1043A000EF0121968491853709F461C058F4843770
:1043B00008F04EC0843008F06AC08130D1F08230FD
:1043C00071F174C0883709F45DC050F4863709F480
:1043D00055C0873709F06AC08E2D0E94AD2454C0A5
:1043E0009CE7980F903708F061C08F770E94B61A4B
:1043F00050C08F010E5F1F4FFE01849190E2980F15
:10440000983050F48770FD2D01C0FF0F8A95EAF7B0
:104410008F2F0E94B32414C00E944B1A13C08F0127
:104420000E5F1F4FFE01C49180E28C0F883060F454
:10443000C7708D2D01C0880FCA95EAF70E94B92474
:104440000E94E424E80125C08C2F0E94B61AFACFFE
:104450009F012E5F3F4FFE01C491CC2369F08FE98D
:104460009FE00197F1F700C00000C150F6CF9F0117
:104470002E5F3F4FFE01F490E9010BC00E949D2486
:10448000E82E07C00E94B0240E94E42402C00E94CB
:104490004B1A8F2D882341F0EFE9FFE03197F1F7B8
:1044A00000C000008150F6CFFE017ACFDF91CF919E
:1044B0001F910F91FF90EF90DF90089560938A0312
:1044C00070938B0380938C0390938D030C946525DC
:1044D000089560938E0370938F038093900390935D
:1044E00091030C9464250F931F9300918E031091F8
:1044F0008F032091900330919103602B712B822BBD
:10450000932B60938E0370938F038093900390930B
:1045100091031F910F910C9464250F931F930091A9
:104520008E0310918F0320919003309191036023AB
:1045300071238223932360938E0370938F03809360
:104540009003909391031F910F910C9464250F9306
:104550001F9300918E0310918F032091900330914F
:104560009103602771278227932760938E037093AE
:104570008F0380939003909391031F910F910C945C
:10458000642560E070E0CB010C945E220F931F93D2
:1045900041E050E060E070E08A019B0104C0000F40
:1045A000111F221F331F8A95D2F7C901B8011F912D
:1045B0000F910C945E220F931F9341E050E060E056
:1045C00070E004C0440F551F661F771F8A95D2F70D
:1045D00080918A0390918B03A0918C03B0918D03FD
:1045E0008A019B01082B192B2A2B3B2BC901B801EF
:1045F0001F910F910C945E220F931F9341E050E0A6
:1046000060E070E004C0440F551F661F771F8A9555
:10461000D2F7409550956095709580918A0390915E
:104620008B03A0918C03B0918D038A019B01082319
:1046300019232A233B23C901B8011F910F910C9420
:104640005E220F931F9341E050E060E070E004C0F1
:10465000440F551F661F771F8A95D2F780918A03F2
:1046600090918B03A0918C03B0918D038A019B01E3
:10467000082719272A273B27C901B8011F910F9145
:104680000C945E220F931F9300918A0310918B0369
:1046900020918C0330918D03602B712B822B932BF7
:1046A0001F910F910C945E220F931F9300918A0328
:1046B00010918B0320918C0330918D036023712323
:1046C000822393231F910F910C945E220F931F93CB
:1046D00000918A0310918B0320918C0330918D03FC
:1046E00060277127822793271F910F910C945E22D8
:1046F00008958F929F92AF92BF92DF92EF92FF92B6
:104700000F931F93CF93DF9300D000D01F92CDB7AC
:10471000DEB76B837C838D838A018C819D81892B9D
:1047200021F01F3F29F44F3F19F480E090E04CC086
:104730008B818823C9F180908E0390908F03A09085
:104740009003B090910380918A0390918B03A09184
:104750008C03B0918D03882A992AAA2ABB2A8FE15B
:10476000E82EF12CD501C4010E2C04C0B695A795F6
:10477000979587950A94D2F780FF07C0DE2CB80181
:104780008E2D0E949E26019729F481E0E81AF108F7
:1047900048F7D12C88E0189FF0011124E00FF11D9B
:1047A000E65BFC4FD08209C088E0189FF00111241D
:1047B000E00FF11DE65BFC4FD08009831A8369810D
:1047C0007A818D2D0E949E260F900F900F900F9052
:1047D0000F90DF91CF911F910F91FF90EF90DF909D
:1047E000BF90AF909F908F90089590912001992352
:1047F00021F090912101911109C020912201309165
:104800002301F90132969FEF40E030C0982F969532
:10481000969596959F31A0F4E0912201F0912301A5
:10482000E90FF11D877021E030E0A90102C0440FBB
:10483000551F8A95E2F7CA019181892B81830895DA
:104840009091B70390FF23C01F928F938AEF96E059
:104850009F938F930E94D8070F900F900F900F9007
:1048600008959F3F39F04F5F4E3141F051915813F9
:10487000F8CF0DC05111F7CF942FF5CF9F3F39F0EE
:10488000F901E90FF11D97FDFA95828308950895C6
:1048900090912001992321F090912101911109C05B
:1048A0002091220130912301F9013296205E3F4F81
:1048B00030C0982F9695969596959F31A8F4E091E3
:1048C0002201F0912301E90FF11D877021E030E012
:1048D000A90102C0440F551F8A95E2F7CA018095CD
:1048E00091818923818308959091B70390FF16C029
:1048F0001F928F938CED96E09F938F930E94D80721
:104900000F900F900F900F9008953196E217F307D4
:1049100029F090819813F9CF1082F7CF089581E0A4
:1049200090E0E0912201F0912301E80FF91F10823D
:10493000019680329105A9F708958091B6030895F4
:104940009091B603892B8093B6030895809590913A
:10495000B60389238093B60308958093B603089520
:104960001092B60308959091B503892B8093B503F7
:10497000089580959091B50389238093B503089598
:104980001092B5030895809394030E94DB259093C1
:1049900093038093920308951092940310929303CB
:1049A0001092920308958091220190912301FC01BD
:1049B00031969C01205E3F4F80E0919191118F5F75
:1049C000E217F307D1F70895E0912201F091230156
:1049D0008091B6038083E0912201F09123019081C0
:1049E0008091B503892B8083809194038823D9F12A
:1049F0000E94DB2520919203309193038217930745
:104A000048F00E94DB252091920330919303821B92
:104A1000930B0AC00E94DB252091920330919303EF
:104A200020953095820F931F8C32914070F08091C9
:104A3000B70380FF08C088E197E09F938F930E949F
:104A4000D8070F900F900E94CC24E0912201F091A2
:104A50002301908180919403892B80830E94D32429
:104A600081110E94CC2480912201909123010C9409
:104A70007D189093A1018093A00108958295982FAD
:104A80009C7C392F36953695282F237344E0249F3C
:104A9000C0011124932F982B292F2A7A2695892F2C
:104AA0008575880F822B08950895CF93DF9300D0EA
:104AB00000D01F92CDB7DEB70F900F900F900F90E0
:104AC0000F90DF91CF910895089508950C94D41913
:104AD0008091CD03843021F11092B80320E488E165
:104AE00090E00FB6F894A895809360000FBE2093D5
:104AF000600083B7817F846083BF83B7816083BF99
:104B00007894889583B78E7F83BF0FB6F894A89565
:104B100080916000886180936000109260000FBEF9
:104B20000895CF930E94F9080E941F080E94FB0875
:104B3000C0E08C2F0E94F008811104C0CF5FC83004
:104B4000C1F701C081E0CF9108950E94D6190C945D
:104B5000381E1F920F920FB60F9211248F939F93BE
:104B6000AF93BF938091B803811113C08091B903B3
:104B70009091BA03A091BB03B091BC034196A11DD3
:104B8000B11D8093B9039093BA03A093BB03B09374
:104B9000BC03BF91AF919F918F910F900FBE0F906B
:104BA0001F90189582E084BD93E095BD9AEF97BD64
:104BB00080936E0008952FB7F8948091B903909177
:104BC000BA03A091BB03B091BC032FBF08952FB7C8
:104BD000F8946091B9037091BA038091BB039091EE
:104BE000BC032FBF0895CF92DF92EF92FF920F93F5
:104BF0001F932FB7F8944091B9035091BA03609175
:104C0000BB037091BC032FBF6A017B01EE24FF241C
:104C10008C0120E030E0C016D106E206F30610F465
:104C2000415051099A01281B390BC9011F910F915D
:104C3000FF90EF90DF90CF900895CF92DF92EF92A8
:104C4000FF920F931F932FB7F894C090B903D090A1
:104C5000BA03E090BB03F090BC032FBF970186011D
:104C6000061B170B280B390BC616D706E806F906E4
:104C700018F0C901B80106C0C901B8016150710935
:104C8000810991091F910F91FF90EF90DF90CF90D4
:104C900008951F920F920FB60F9211248F939F9336
:104CA000AF93BF938091B9039091BA03A091BB03D6
:104CB000B091BC030196A11DB11D8093B9039093DF
:104CC000BA03A093BB03B093BC03BF91AF919F9174
:104CD0008F910F900FBE0F901F9018950E94851511
:104CE000F8942FEF87EA91E6215080409040E1F759
:104CF00000C0000087E090EBDC018093D603909326
:104D0000D703A093D803B093D9039CE088E10FB6F2
:104D1000F894A895809360000FBE90936000FFCF39
:104D200028E0929FF0011124E80FF11DEE58FE4F8C
:104D30009491892F8F7092959F700895CF93C82F6B
:104D4000CB010E949026282F30E080E1989FA0019F
:104D50001124422B532B4038510519F480E090E088
:104D600015C09770E92FF0E088E0C89FE00DF11DB5
:104D7000112484E0EE0FFF1F8A95E1F7E20FF31F85
:104D8000EE0FFF1FE050F84985919491CF9108955F
:104D900080E090E0089508958091BF0380FF0BC0EC
:104DA0006091270185E0689FB00111247595679592
:104DB000759567952BC081FF09C06091270185E03B
:104DC000689FB00111247595679520C082FF07C0C8
:104DD0006091270185E0689FB001112417C0909170
:104DE000C0039923D1F060912601961788F720918E
:104DF000270185E0289F90011124929FA001939F95
:104E0000500D112470E0CA010E94B42E6038710563
:104E100040F46115710539F002C065E070E0862F3D
:104E200008958FE7089581E008958091BF0380FF82
:104E300008C06091250170E0759567957595679537
:104E400021C081FF06C06091250170E075956795CE
:104E500019C082FF04C06091250170E010C09091DC
:104E6000C0039923C1F0609124019617A0F78091A7
:104E70002501899FC001112470E00E94B42E603882
:104E8000710528F46115710521F0862F08958FE7CB
:104E9000089581E0089561E070E0F4CF803F21F44F
:104EA0000E94CC26819504C0813F29F40E94CC2623
:104EB0008093C3030895823F21F40E94CC268195FC
:104EC00004C0833F29F40E94CC268093C203089536
:104ED000893F19F40E94152705C08A3F31F40E94CA
:104EE000152781958093C40308958B3F21F40E9478
:104EF0001527819504C08C3F29F40E9415278093C3
:104F0000C5030895843F21F48091C103816017C0D7
:104F1000853F21F48091C103826011C0863F21F456
:104F20008091C10384600BC0873F21F48091C1034D
:104F3000886005C0883F31F48091C103806180930F
:104F4000C10308958D3F21F48091BF0381600BC0A0
:104F50008E3F21F48091BF03826005C08F3F29F40A
:104F60008091BF0384608093BF030895803F39F42C
:104F70008091C30387FF6CC01092C30369C0813F57
:104F800029F48091C3031816BCF362C09091C20348
:104F9000823F29F497FF5CC01092C20359C0833F3F
:104FA00019F41916CCF354C0893F41F48091C4031D
:104FB00018160CF04DC01092C4034AC08A3F29F461
:104FC0008091C40387FF44C0F6CF8B3F39F48091B2
:104FD000C50387FF3DC01092C5033AC08C3F29F43A
:104FE0008091C5031816BCF333C0843F21F480912F
:104FF000C1038E7F17C0853F21F48091C1038D7F4F
:1050000011C0863F21F48091C1038B7F0BC0873F85
:1050100021F48091C103877F05C0883F31F48091DE
:10502000C1038F7E8093C10313C08D3F21F4809113
:10503000BF038E7F0BC08E3F21F48091BF038D7F15
:1050400005C08F3F29F48091BF038B7F8093BF03FE
:105050008091C20381110EC08091C30381110AC0E7
:105060008091C403811106C08091C503811102C0E3
:105070001092C00308958091B70383FF7EC081E53D
:1050800097E00E943F078091C1031F928F938CE4A9
:1050900097E09F938F930E94D8078AE497E00E943D
:1050A0003F078091C203282F082E000C330B3F933B
:1050B0008F9387E497E09F938F930E94D80785E4AE
:1050C00097E00E943F078091C303282F082E000C11
:1050D000330B3F938F9382E497E09F938F930E94CB
:1050E000D80780E497E00E943F078091C403282FEF
:1050F000082E000C330B3F938F938DE397E09F9323
:105100008F930E94D8078BE397E00E943F0780911E
:10511000C503282F082E000C330B3F938F9388E391
:1051200097E09F938F930E94D80785E397E00E94B2
:105130003F078091C0031F928F9382E397E09F9374
:105140008F930E94D80780E397E00E943F078091E9
:10515000BF031F928F938DE297E09F938F930E94DE
:10516000D8078AE297E00E943F078DB79EB74C961A
:105170000FB6F8949EBF0FBE8DBF81EC93E00E94E6
:10518000C6180E94DB259093BE038093BD0308954B
:105190001F93CF93DF938091BD039091BE030E9434
:1051A000F325AC019091C003992321F020912801AF
:1051B00030E006C0209129018AE0289F9001112447
:1051C0004217530708F485C08091C203C091C303FE
:1051D000D091C4031091C503811107C0C11175C0DE
:1051E000D11173C0111171C074C09F3F19F09F5F3E
:1051F0009093C003181624F40E94CC268093C20317
:105200008091C20387FF05C00E94CC2681958093C0
:10521000C2031C1624F40E94CC268093C303809101
:10522000C30387FF05C00E94CC2681958093C303EA
:105230006091C203662331F1C091C303CC2311F105
:10524000062E000C770B880B990B0E949B2D23E3F5
:1052500033E343E35FE30E94FF2D0E94632D6093DD
:10526000C2036C2FCC0F770B880B990B0E949B2DE0
:1052700023E333E343E35FE30E94FF2D0E94632DAA
:105280006093C3031D1624F40E9415278093C40362
:105290008091C40387FF05C00E94152781958093E4
:1052A000C403111624F40E9415278093C50380912E
:1052B000C50387FF05C00E94152781958093C5030C
:1052C000DF91CF911F910C943B289F3F09F08FCF26
:1052D00097CFDF91CF911F910895E1ECF3E085E046
:1052E000DF011D928A95E9F71092C0031092BF0367
:1052F000089584E799E00E943F071F9281E08F9311
:105300001F9285E08F9386E299E09F938F930E948E
:10531000D8070F900F900F900F900F900F90089557
:105320008330E9F128F4813061F0823009F1089589
:10533000853009F462C008F449C0863009F474C0AD
:10534000089580912901262F30E0280F311D2F3F2D
:10535000310524F4680F6093290103C08FEF809317
:105360002901809129011F928F938FE598E072C0E7
:1053700080912801262F30E0280F311D2F3F310565
:1053800024F4680F6093280103C08FEF80932801F5
:10539000809128011F928F938DE498E05BC08091EB
:1053A0002701262F30E0280F311D2F3F310524F42F
:1053B000680F6093270103C08FEF809327018091CE
:1053C00027011F928F938AE398E044C080912601C1
:1053D000262F30E0280F311D2F3F310524F4680FB0
:1053E0006093260103C08FEF8093260180912601F0
:1053F0001F928F9385E298E02DC080912501262F82
:1054000030E0280F311D2F3F310524F4680F6093E1
:10541000250103C08FEF80932501809125011F9204
:105420008F938CE098E016C080912401262F30E005
:10543000280F311D2F3F310524F4680F609324019C
:1054400003C08FEF80932401809124011F928F93DA
:1054500081EF97E09F938F930E94D8070F900F9052
:105460000F900F900895833081F128F4813059F026
:105470008230D1F00895853009F449C0B8F1863002
:1054800009F456C0089580912901681720F4861BFD
:105490008093290102C010922901809129011F9255
:1054A0008F9382EE97E054C080912801681720F412
:1054B000861B8093280102C0109228018091280148
:1054C0001F928F9380ED97E043C08091270168176A
:1054D00020F4861B8093270102C01092270180913F
:1054E00027011F928F938DEB97E032C080912601A8
:1054F000681720F4861B8093260102C010922601B3
:10550000809126011F928F9388EA97E021C08091B5
:105510002501681720F4861B8093250102C0109294
:105520002501809125011F928F938FE897E010C08D
:1055300080912401681720F4861B8093240102C007
:1055400010922401809124011F928F9384E797E0A9
:105550009F938F930E94D8070F900F900F900F90FA
:105560000895CF93C82F1F928F9389E79AE09F9356
:105570008F930E94D80781E090E0A0E0B0E0BC01EA
:10558000CD0104C0660F771F881F991FCA95D2F7F7
:105590000E9469220F900F900F900F90CF910C9462
:1055A000381ECF938732A8F58E3108F02BC1803199
:1055B00009F49FC0F8F4873009F464C0A8F4863079
:1055C00009F024C18091B703817F8E7F8093B70358
:1055D0008EE79AE00E943F0782E69DE00E943F0727
:1055E00081E08093C7034CC08B30F1F18E3009F419
:1055F0006CC00CC1863109F4B0C020F4813109F4CB
:10560000EDC004C1893109F491C08B3109F449C05E
:10561000FDC0883349F150F4893209F4F1C0853373
:1056200009F4EEC0873209F0F1C0EAC0833409F40E
:10563000E7C028F48A3308F4E9C08953E4C0883409
:1056400009F0E4C00E94381E81E59DE00E943F07FA
:105650002FEF83ED90E3215080409040E1F700C0B0
:1056600000000E946E260CC085EA9AE05CC088E3C8
:105670009DE00E943F078091B70381608093B7034C
:10568000C1E0C9C08091B703C82FC17080FFEFCFC0
:1056900084E49DE00E943F078091B703817F8E7F65
:1056A0003DC09091B70391FBCC27C0F981E0C8279A
:1056B000892FC0FB81F98093B703CC2319F08BE2CB
:1056C0009DE027C08DE19DE02EC09091B70392FB35
:1056D000CC27C0F981E0C827892FC0FB82F98093CD
:1056E000B703CC2319F08EE09DE013C08EEF9CE051
:1056F0001AC09091B70393FBCC27C0F981E0C8276B
:10570000892FC0FB83F98093B703CC2351F082EF3C
:105710009CE00E943F078091B70381608093B703AC
:105720007AC085EE9CE00E943F07AACF86ED9CE000
:105730000E943F0789EA9CE00E943F0782E79CE0C5
:105740000E943F078BE49CE00E943F0781E09CE0C1
:105750000E943F0783ED9BE0E6CF85EC9BE00E9433
:105760003F070E9471181F928F938BEA9BE09F93D3
:105770008F930E94D807809120011F928F9384E914
:105780009BE09F938F930E94D807809102031F9202
:105790008F9381E89BE09F938F930E94D80780911D
:1057A00021011F928F938EE69BE09F938F930E941F
:1057B000D8070E94E7259F938F937F936F9387E588
:1057C0009BE09F938F930E94D8078DB79EB7469614
:1057D0000FB6F8949EBF0FBE8DBF52CF0E94381EE9
:1057E000C091210181E0C827C0932101CC2329F079
:1057F0008DE49BE00E943F070EC082E49BE093CFC4
:1058000080E001C08D510E94B12A3ACF80E49BE034
:105810000E943F07C0E08C2FCF910895CF93C82FEF
:105820008091C703813071F020F0823009F44BC0C1
:1058300042C1E0912201F09123018081823209F07E
:105840003CC107C0E0912201F091230180818232A6
:1058500061F48C2F0E943B0C811104C08C2F0E949C
:10586000D12A2FC081E090E02CC08C2F0E946F0EB7
:10587000811126C0C431E1F070F4CB3081F0C03129
:10588000D1F40E94792981E79AE00E943F0782E0E3
:105890008093C70315C0C93259F0C83361F48EE74D
:1058A0009AE00E943F0785E79AE00E943F0708C000
:1058B0001092C70304C18FE69AE00E943F07FFC021
:1058C00081E08170FEC0C43228F5CE3108F0C1C03D
:1058D000CB30A1F1D0F4C73009F0D3C08EE1809372
:1058E000290182E3809328018AE08093270184E1E3
:1058F0008093260188E08093250188E2809324012B
:1059000085E199E00E943F07BFC0C33149F1C4312E
:10591000C1F0B7C0CB3409F4A9C028F4C93289F06A
:10592000C83361F0AEC0C13509F49EC0C23509F478
:1059300099C0CE3409F0A5C06AE09EC00E947929C2
:10594000A3C08091C603882319F01092C6039CC09F
:1059500082E299E00E943F0781E08093C703B1C0D3
:105960008CEF98E00E943F078AEE98E00E943F0784
:10597000809129011F928F9387EE98E09F938F93D8
:105980000E94D80785EE98E00E943F0783ED98E0DB
:105990000E943F07809128011F928F9380ED98E02D
:1059A0009F938F930E94D8078EEC98E00E943F0748
:1059B0008FEB98E00E943F07809127011F928F9301
:1059C0008CEB98E09F938F930E94D8078AEB98E026
:1059D0000E943F0789EA98E00E943F0780912601D4
:1059E0001F928F9386EA98E09F938F930E94D80727
:1059F00084EA98E00E943F078FE898E00E943F0702
:105A0000809125011F928F938CE898E09F938F934C
:105A10000E94D8078AE898E00E943F0783E798E051
:105A20000E943F07809124011F928F9380E798E0A6
:105A30009F938F930E94D8078EE698E00E943F07BD
:105A40008DB79EB748960FB6F8949EBF0FBE8DBF18
:105A50001BC0CE51EC2FF0E0EA56FE4F80818093C0
:105A6000C60312C061E003C061E006C06AE0809135
:105A7000C6030E94902908C08091C6030E94332A61
:105A800003C083E199E013C08091C603882369F0C5
:105A90001F928F938DE099E09F938F930E94D80778
:105AA0000F900F900F900F9004C08AE099E00E9431
:105AB0003F0781E006C01092C70380E002C080E08B
:105AC00000CFCF9108950E946A2D6894B1110C9473
:105AD000F92D08950E94DE2D88F09F5798F0B92F78
:105AE0009927B751B0F0E1F0660F771F881F991F13
:105AF0001AF0BA95C9F714C0B13091F00E94F82D90
:105B0000B1E008950C94F82D672F782F8827B85F9F
:105B100039F0B93FCCF3869577956795B395D9F76A
:105B20003EF490958095709561957F4F8F4F9F4F74
:105B30000895E89409C097FB3EF490958095709580
:105B400061957F4F8F4F9F4F9923A9F0F92F96E9C9
:105B5000BB279395F695879577956795B795F1113E
:105B6000F8CFFAF4BB0F11F460FF1BC06F5F7F4FDB
:105B70008F4F9F4F16C0882311F096E911C07723ED
:105B800021F09EE8872F762F05C0662371F096E8F6
:105B9000862F70E060E02AF09A95660F771F881FC5
:105BA000DAF7880F9695879597F9089557FD9058DD
:105BB000440F551F59F05F3F71F04795880F97FBD1
:105BC000991F61F09F3F79F087950895121613068B
:105BD0001406551FF2CF4695F1DF08C016161706BA
:105BE0001806991FF1CF86957105610508940895EF
:105BF000E894BB2766277727CB0197F908950E9481
:105C0000122E0C94832E0E94752E38F00E947C2E4A
:105C100020F0952311F00C946C2E0C94722E11240C
:105C20000C94F92D0E94D62D70F3959FC1F3950F1A
:105C300050E0551F629FF001729FBB27F00DB11D10
:105C4000639FAA27F00DB11DAA1F649F6627B00DA0
:105C5000A11D661F829F2227B00DA11D621F739F89
:105C6000B00DA11D621F839FA00D611D221F749F97
:105C70003327A00D611D231F849F600D211D822FDE
:105C8000762F6A2F11249F5750409AF0F1F0882305
:105C90004AF0EE0FFF1FBB1F661F771F881F915032
:105CA0005040A9F79E3F510580F00C946C2E0C9447
:105CB000F92D5F3FE4F3983ED4F386957795679589
:105CC000B795F795E7959F5FC1F7FE2B880F911D5C
:105CD0009695879597F9089597F99F6780E870E002
:105CE00060E008959FEF80EC089500240A94161652
:105CF000170618060906089500240A9412161306BA
:105D0000140605060895092E0394000C11F4882347
:105D100052F0BB0F40F4BF2B11F460FF04C06F5F63
:105D20007F4F8F4F9F4F0895991B79E004C0991FB3
:105D3000961708F0961B881F7A95C9F780950895E5
:105D4000AA1BBB1B51E107C0AA1FBB1FA617B707A1
:105D500010F0A61BB70B881F991F5A95A9F78095BD
:105D60009095BC01CD01089597FB072E16F4009481
:105D700007D077FD09D00E94A02E07FC05D03EF485
:105D8000909581959F4F0895709561957F4F0895E7
:105D9000A1E21A2EAA1BBB1BFD010DC0AA1FBB1F2F
:105DA000EE1FFF1FA217B307E407F50720F0A21BA1
:105DB000B30BE40BF50B661F771F881F991F1A940E
:105DC00069F760957095809590959B01AC01BD0138
:105DD000CF010895EE0FFF1F0590F491E02D099477
:045DE000F894FFCF65
:105DE4008509880989098A098B098109050AEB094A
:105DF40084098C090A010111F211CF119B11671159
:105E0400010195032808140A321E524E2D34320023
:105E14004C554641004F4646004F4E00434F4E4EB0
:105E240000506F776572656400556E6174746163C8
:105E34006865640044656661756C740041646472ED
:105E4400657373656400436F6E6669677572656434
:105E5400003F0053757370656E64656400404D3691
:105E640022394406F705C1059F056605D904F204E5
:105E74000B0524054405010203040506070809006F
:106800000000000000000000040005000600070072
:10681000080009000A000B000C000D000E000F001C
:1068200010001100120013001400150016001700CC
:10683000180019001A001B001C001D001E001F007C
:10684000200021002200230024002500260027002C
:106850002800000035002B002C002D002E002F00FA
:1068600030002A00000033003400290036003700D1
:106870003800E00000000000000000000000000000
:106880000000000000000000000000000000000008
:1068900000000000000000000000000000000000F8
:1068A00000000000000000000000000000000000E8
:1068B00000000000000000000000000000000000D8
:1068C00000000000000000000000000000000000C8
:1068D00000000000000000000000000000000000B8
:1068E0000000000000000000310000000000000077
:1068F0000000E100E200E300F1A1E500E600E700AE
:106900000000000000000000EA4401000100E24431
:106910000100010001005500460054004A004B00F0
:10692000560057004700480001000100E9440100FB
:106930000100010001000100010001003A003B00DC
:106940003C003D003E003F0040004100420043004B
:10695000580000004C00390001004400450052007E
:1069600001000100000050004F0081404D004E002A
:1069700051000100000000000000000000000000C5
:106980000000000000000000000000000000000007
:1069900000000000000000000000000000000000F7
:1069A00000000000000000000000000000000000E7
:1069B00000000000000000000000000000000000D7
:1069C00000000000000000000000000000000000C7
:1069D00000000000000000000000000000000000B7
:1069E000000000000000000049000000000000005E
:1069F0000000010001000100010001000100010090
:00000001FF
